:10000000B7C00000D2C00000D0C00000CEC00000C9
:10001000CCC00000CAC00000C8C00000C6C00000BC
:10002000C4C00000C2C00000C0C0000042C7000041
:10003000E2C70000BAC00000B8C00000B6C00000AF
:10004000B4C00000B2C00000B0C00000AEC00000EC
:10005000ACC00000AAC00000A8C00000A6C00000FC
:10006000A4C00000A2C00000A0C000009EC000000C
:100070009CC0000030034C005500460041002000A9
:10008000430044004300200061006E006400200033
:100090004D006F007500730065002000440065008E
:1000A0006D006F00000018034400650061006E00E1
:1000B0002000430061006D006500720061000000D7
:1000C0000403090409025F00030100C032080B00A9
:1000D00002020201000904000001020201000524DD
:1000E000001001042402060524060001070582030E
:1000F0000800FF09040100020A00000007050402CD
:100100001000050705830210000509040200010321
:10011000010200092111010001223A0007058103B3
:1001200008000512011001EF020108EB0362200133
:10013000000102DC0105010902A1010901A100057C
:1001400009190129031500250195037501810295FF
:10015000017505810105010930093116FFFF2601EE
:100160000036FFFF460100950275088106C0C000F9
:1001700011241FBECFEFD2E0DEBFCDBF11E0A0E063
:10018000B1E0E4E5FBE102C005900D92A433B107B4
:10019000D9F721E0A4E3B1E001C01D92A434B20775
:1001A000E1F70E94600A0C94A80D2ACF292F33276B
:1001B00023303105C9F040F42130310509F438C04D
:1001C0002230310561F006C02132310539F1223289
:1001D000310549F180E090E020E030E032C08FE569
:1001E00090E024EC30E02DC099278130910551F04A
:1001F00018F0029769F021C0E0ECF0E0849190E003
:100200009F011FC0E6EAF0E0849190E09F0119C0D1
:10021000E4E7F0E0849190E09F0113C089E090E072
:1002200023E131E00EC08AE390E025E331E009C02C
:1002300082E190E023E231E004C080E090E020E041
:1002400030E0FA01318320830895CF93DF93EC01EE
:10025000FC0170968BE0DF011D928A95E9F782E040
:100260008C83898783E08E8761E0CE01019636D545
:10027000882351F061E0CE01069630D5882321F025
:1002800061E0CE010B962AD5DF91CF910895FC0154
:1002900090913B019430C9F484899589A689B789E6
:1002A000892B8A2B8B2B99F0CB0121812F702093E6
:1002B000E900FB0101900020E9F73197BF01681BBD
:1002C000790B40E050E07FC3089582E0089582E01A
:1002D0000895CF93FC0190913B01943019F58489E6
:1002E0009589A689B789892B8A2B8B2BE9F0818187
:1002F0008F708093E9008091F2008823B9F0E8EED6
:10030000F0E0908180818E778083C92FC07295FD47
:100310000FC051D581110EC0E8EEF0E080818E77DC
:10032000808309C0C2E007C0C2E005C0C0E003C0CE
:10033000C0E001C0C82F8C2FCF910895FC0190918F
:100340003B01943091F484899589A689B789892BDA
:100350008A2B8B2B51F081818F708093E9008091E3
:10036000E80080FF02C0CF01B4CF0895FC01909156
:100370003B019430F9F484899589A689B789892B42
:100380008A2B8B2BD1F086818F708093E90080912E
:10039000E80082FF15C08091F20090E0009731F4F0
:1003A000E8EEF0E020812B77208308958091F20021
:1003B00090E0089580E090E0089580E090E0089556
:1003C00080E090E0089520913B01243039F5FC0154
:1003D0004489558966897789452B462B472B09F136
:1003E00086818F708093E9008091E80082FF1CC0B5
:1003F0008091F200882321F02091F10030E002C0CA
:100400002FEF3FEF8091F200811111C0E8EEF0E094
:1004100080818B778083822F932F08958FEF9FEFBA
:1004200008958FEF9FEF08958FEF9FEF0895822F2C
:10043000932F08950895CF93DF93FC019091E800E6
:1004400093FF98C08091400190914101208130E05C
:100450008217930709F08EC0EF0180913D01813230
:1004600059F018F48032C1F185C0823209F461C0BC
:10047000833209F471C07EC080913C01813A09F059
:1004800079C0E8EEF0E08081877F80838091E8008A
:1004900080FFFCCF8C899D89AE89BF89E1EFF0E0B8
:1004A0008083492F5A2F6B2F77274083AD01662712
:1004B000772740838B2F9927AA27BB278083888D96
:1004C0008083898D80838A8D8083E8EEF0E080814F
:1004D0008E7780834FD44EC080913C01813209F0E9
:1004E00049C0E8EEF0E08081877F808305C080917D
:1004F0003B01882309F43EC08091E80082FFF7CFDA
:10050000E1EFF0E030812081908180813C8B2D8B68
:100510009E8B8F8B8081888F8081898F80818A8F4D
:10052000E8EEF0E080818B77808324D4CE0182DFF7
:1005300021C080913C018132E9F4E8EEF0E0808155
:10054000877F808317D480913E0190913F01998BE2
:10055000888BCE01FBD70EC080913C01813251F4D3
:10056000E8EEF0E08081877F808304D460913E01D3
:10057000CE0160DFDF91CF9108953F924F925F925D
:100580006F927F928F929F92AF92BF92CF92DF92A3
:10059000EF92FF920F931F93CF93DF9300D01F92A0
:1005A000CDB7DEB76C01EDB6FEB68091E80083FFF3
:1005B0001DC12091400130914101F601808190E000
:1005C0002817390709F012C180913D01833009F4E1
:1005D000A8C030F4813071F0823009F4EBC006C15C
:1005E0008A3009F4CBC08B3009F4B4C0893009F0EB
:1005F000FDC050C080913C01813A09F0F7C0ADB612
:10060000BEB61A821982ECE3F1E0828173808B839B
:100610007A94F601408550E08DB79EB7841B950B08
:100620000FB6F8949EBF0FBE8DBFEDB7FEB73196E3
:100630004F0160E070E0CF01A0D78E010F5F1F4F28
:100640009401472DBE016D5F7F4FC60173D7F60140
:1006500086819781009721F0408550E0B40184D7CE
:100660001092E900E8EEF0E08081877F80838B8143
:1006700081118093F10069817A81C401EDD1E8EEA6
:10068000F0E080818B7780830FB6F894BEBE0FBEFA
:10069000ADBEACC080913C01813209F0A7C06DB6FF
:1006A0007EB6ECE3F1E00681178142805380342C62
:1006B0005A948DB79EB7801B910B0FB6F8949EBFCE
:1006C0000FBE8DBFEDB7FEB731964F010F2EF8EE7E
:1006D000AF2EB12CF02DF5018081877F8083B8018A
:1006E000C4011DD2F50180818E778083442019F0EA
:1006F00081E090E002C080E090E021E030E0311045
:1007000002C020E030E0280D391D081B190B452DD3
:10071000642DC6011AD70FB6F8947EBE0FBE6DBE0B
:1007200065C080913C01813A09F060C0E8EEF0E0DC
:100730008081877F80838091E80080FFFCCFF60175
:1007400081858093F100E8EEF0E080818E778083F0
:1007500011D34CC080913C01813209F047C0E8EED2
:10076000F0E08081877F808305D390913E0181E016
:10077000911101C080E0F601818738C080913C0171
:100780008132A1F5E8EEF0E08081877F8083F2D2AC
:1007900080913E0190913F0188270024880F991F86
:1007A000001C880F991F001C892F902DF60195873A
:1007B00084871CC080913C01813AC1F4E8EEF0E0EE
:1007C0008081877F80838091E80080FFFCCFF601E5
:1007D0008485958596958795969587958093F10064
:1007E000E8EEF0E080818E778083C4D20FB6F89473
:1007F000FEBE0FBEEDBE0F900F900F90DF91CF9118
:100800001F910F91FF90EF90DF90CF90BF90AF902E
:100810009F908F907F906F905F904F903F90089542
:10082000FC01399627E0DF011D922A95E9F721E0C6
:10083000FC01218724EF31E03587248723E02483DE
:1008400061E001964BC208955F926F927F928F9202
:100850009F92AF92BF92CF92DF92EF92FF920F934F
:100860001F93CF93DF9300D01F92CDB7DEB77C01EB
:10087000ADB6BEB680913B01843009F08CC0F70163
:10088000228533858091E4009091E500281739078F
:1008900009F481C081818F708093E9008091E80024
:1008A00085FF79C08DB69EB6408550E08DB79EB766
:1008B000841B950B0FB6F8949EBF0FBE8DBFEDB78E
:1008C000FEB731966F011B821A82198260E070E0D8
:1008D000CF0153D68E010F5F1F4F960140E0BE013E
:1008E0006D5F7F4FC70126D6682EF70184859585F9
:1008F000892B31F086859785892B21F080E003C014
:1009000080E001C081E08170782EF70106811781B7
:100910000115110589F049815A81B801C60117D620
:1009200055245394892B09F4512CF701408550E04C
:10093000B601C80119D601C0512C89819A81892B31
:10094000F1F0611004C0511002C07720C1F0F7012E
:10095000848595859787868781818F708093E9004C
:100960008B8181118093F10069817A8140E050E0B0
:10097000C60129D0E8EEF0E080818E7780838091F7
:10098000E4009091E500F701938782870FB6F89411
:100990009EBE0FBE8DBE0FB6F894BEBE0FBEADBEDE
:1009A0000F900F900F90DF91CF911F910F91FF90BB
:1009B000EF90DF90CF90BF90AF909F908F907F90FF
:1009C0006F905F900895CF92DF92EF92FF920F9316
:1009D0001F93CF93DF938C01EB016A01ECD181115E
:1009E00032C0C114D10439F0F60180819181C81B55
:1009F000D90B080F191FE12CF12C22C08091E800BF
:100A000085FD15C0E8EEF0E090819E779083C114DB
:100A1000D10449F0F60180819181E80EF91EF1823E
:100A2000E08285E010C0C7D1882351F00CC0F801E6
:100A300081918F018093F1002197FFEFEF1AFF0A58
:100A40002097E1F680E0DF91CF911F910F91FF9009
:100A5000EF90DF90CF9008952091420130914301B3
:100A60002617370758F06115710539F4E8EEF0E004
:100A700020812E7720839B0101C09B01E82FF92F55
:100A800040E02BC080913B018823E9F18530E9F1FA
:100A90008091E80083FD3BC08091E80082FD2DC07D
:100AA0008091E80080FF19C08091F20090E006C0BC
:100AB00041914093F10021503109019621153105F2
:100AC00019F088309105A0F341E0089709F040E063
:100AD000A8EEB0E08C918E778C932115310591F6BC
:100AE0004111D0CF0AC080913B01882391F085301D
:100AF00091F08091E80083FD10C08091E80082FFB2
:100B0000F2CF80E0089582E0089583E0089581E0C7
:100B1000089582E0089583E0089581E008956115C5
:100B2000710529F4E8EEF0E020812B772083E82F8F
:100B3000F92F20C080913B01882361F1853061F15C
:100B40008091E80083FD2AC08091E80082FF12C0F6
:100B500005C08091F10081936150710961157105A3
:100B600021F08091F2008111F4CFA8EEB0E08C91D9
:100B70008B778C9361157105E9F606C080913B0176
:100B8000882371F0853071F08091E80080FFF6CF06
:100B900080E0089582E0089583E0089581E008955B
:100BA00082E0089583E0089520914201309143014D
:100BB0002617370758F06115710539F4E8EEF0E0B3
:100BC00020812E7720839B0101C09B01E82FF92F04
:100BD00040E02EC080913B01882309F43FC085305E
:100BE00009F43EC08091E80083FD3CC08091E8009C
:100BF00082FD2EC08091E80080FF1AC08091F20033
:100C000090E007C044914093F100319621503109A2
:100C100001962115310519F08830910598F341E0CE
:100C2000089709F040E0A8EEB0E08C918E778C93A5
:100C30002115310579F64111CDCF0AC080913B01D4
:100C4000882391F0853091F08091E80083FD10C0F9
:100C50008091E80082FFF2CF80E0089582E008955D
:100C600083E0089581E0089582E0089583E0089587
:100C700081E00895982F29C0292F2F702093E90033
:100C8000981739F07091EC002091ED005091F00030
:100C900003C0242F762F50E021FF16C0EBEEF0E0CA
:100CA00030813E7F3083ADEEB0E03C913D7F3C93A0
:100CB0003081316030837093EC002C935093F000BE
:100CC0002091EE00222344F49F5F9530A8F28F70AC
:100CD0008093E90081E0089580E008950F931F93C9
:100CE000CF93DF93EC01062F10E03CC0E12FF0E042
:100CF000CF01880F991F880F991FE80FF91FEC0F7C
:100D0000FD1F5081552369F19481A181B2816381D6
:100D1000852F8F70853010F5923010F046E001C0BD
:100D200042E028E030E090E003C09F5F220F331FD5
:100D30002A173B07D0F39295907F70E000247695B8
:100D400067950794769567950794762F602D551FC4
:100D50005527551F492B652B8DDF01C080E0882367
:100D600021F01F5F101710F281E0DF91CF911F91EA
:100D70000F91089580913C0188239CF404C08091D8
:100D80003B018823B9F08091E80082FFF8CFE8EEBC
:100D9000F0E080818B778083089580913B018823E8
:100DA00049F08091E80080FFF8CFE8EEF0E0808124
:100DB0008E77808308952091E4003091E50044E629
:100DC00002C09C01452F8091EC00982F917080FD0E
:100DD00090E8903829F48091E80080FF05C01BC09E
:100DE0008091E80082FD19C080913B018823B9F011
:100DF0008530B9F08091EB0085FD15C08091E4004D
:100E00009091E50028173907F1F25FEF540F411177
:100E1000D8CF84E0089580E0089580E0089582E0CE
:100E2000089583E0089581E0089510923B011092A7
:100E30003701109239011092380142E060E080E001
:100E400019DFE1EEF0E080818E7F8083E2EEF0E05A
:100E5000808181608083808188608083E0EEF0E023
:100E600080818E7F808308951ED020D0E8EDF0E051
:100E700080818F77808380818068808380818F7D6F
:100E8000808319BC82E089BD09B400FEFDCFCDCFBF
:100E90000895E3E6F0E080818E7F808381E0809397
:100EA0003A01E2CF08951092E20008951092E10015
:100EB00008951F920F920FB60F9211242F933F9314
:100EC0004F935F936F937F938F939F93AF93BF9352
:100ED000EF93FF938091E10082FF0AC08091E200CE
:100EE00082FF06C0E1EEF0E080818B7F808316D325
:100EF0008091E10080FF15C08091E20080FF11C069
:100F0000E2EEF0E080818E7F80838081806180834B
:100F1000E8EDF0E080818062808319BC10923B0193
:100F2000E7D28091E10084FF2EC08091E20084FF2F
:100F30002AC019BC82E089BD09B400FEFDCFE8EDEE
:100F4000F0E080818F7D8083E1EEF0E080818F7E14
:100F50008083E2EEF0E080818F7E808380818160FB
:100F6000808380913701882321F084E080933B01C6
:100F700009C08091E300882314F483E001C081E07C
:100F800080933B01B4D28091E10083FF23C0809124
:100F9000E20083FF1FC0E1EEF0E08081877F808365
:100FA00082E080933B011092370180818E7F8083A5
:100FB000E2EEF0E080818E7F80838081806180839B
:100FC00042E060E080E056DEE0EFF0E080818860A3
:100FD000808300D2FF91EF91BF91AF919F918F914C
:100FE0007F916F915F914F913F912F910F900FBE25
:100FF0000F901F9018951F920F920FB60F92112409
:10100000EF92FF921F932F933F934F935F936F93B2
:101010007F938F939F93AF93BF93CF93DF93EF9380
:10102000FF93C091E900CF708091EC00982F9170F0
:1010300080FD90E8192F1C2B0F2EF9EEEF2EF12CCE
:10104000F02DF7011082C0EFD0E08881877F888380
:10105000789471D1F7011082888188608883C12FCC
:10106000CF70C083FF91EF91DF91CF91BF91AF918E
:101070009F918F917F916F915F914F913F912F91B0
:101080001F91FF90EF900F900FBE0F901F9018953B
:1010900080913C01803819F0823871F00895809178
:1010A0003801811102C090E001C091E080913901C6
:1010B000882381F092600EC0809140018F7085304E
:1010C000B0F4E9EEF0E080839091EB0095FB992776
:1010D00090F91082E8EEF0E08081877F8083A1EFB5
:1010E000B0E09C931C9280818E77808343CE0895DC
:1010F00080913C018F7119F0823071F008958091D8
:101100003E01813009F03FC090913D01933009F0DC
:1011100080E0809339012FC080913E0181112BC066
:10112000809140018F709FEF980F943060F580930D
:10113000E9009091EB0090FF1EC090913D0193302B
:1011400031F4EBEEF0E080818062808314C0EBEE3E
:10115000F0E090819061908321E030E0A90102C02D
:10116000440F551F8A95E2F7AAEEB0E04C931C920B
:101170008081886080831092E900E8EEF0E0808151
:10118000877F8083F7CD0895CF93C0913E01CF77BD
:10119000E3EEF0E0808180788C2B8083E8EEF0E055
:1011A0008081877F8083E6DD8091E80080FFFCCF2F
:1011B000E3EEF0E0808180688083CC2311F083E04F
:1011C00001C082E080933B01CF910895E8EEF0E00A
:1011D0008081877F8083809137018093F1008081B7
:1011E0008E778083C7CD08950F931F93CF93DF939E
:1011F000CDB7DEB7AA970FB6F894DEBF0FBECDBF4E
:1012000083E08A838AE289833FB7F89490E02EE0F6
:1012100020C0E22FF0E081E280935700E49190FF3C
:1012200003C0E295EF702F5FEF70A92FB0E0AA0F17
:10123000BB1F43E050E04C0F5D1FA40FB51FEA3009
:1012400018F0F0E0F79602C0F0E0F096ED93FC9312
:101250009F5F9431F0F23FBF08EE10E0F80180810B
:10126000877F80836AE270E0CE010196F5DBF801AA
:1012700080818B778083AA960FB6F894DEBF0FBE6D
:10128000CDBFDF91CF911F910F9108950F931F93C1
:10129000CF93DF9300D0CDB7DEB780913E01909120
:1012A0003F018C3D23E0920711F49EDF19C060914D
:1012B000400170914101AE014F5F5F4F0E94D60027
:1012C000009771F008EE10E0F8012081277F20835D
:1012D000BC0189819A8168DCF80180818B778083E9
:1012E0000F900F90DF91CF911F910F9108958091F2
:1012F0003E0190913F0199270297E4F4E8EEF0E077
:101300008081877F808380913E018093370132DD29
:1013100080913701882321F084E080933B0109C04C
:101320008091E300882314F484E001C081E080937D
:101330003B01DFC0089580E0ECE3F1E005C090914F
:10134000F10090838F5F31968830C8F3DFD08091B1
:10135000E80083FF30C0ECE3F1E0908181818530CB
:10136000D1F030F4813089F050F0833071F023C037
:101370008830D1F08930E1F08630E9F410C090383F
:1013800011F09238C1F484DE16C0992311F0923026
:1013900091F4AEDE10C091110EC0F6DE0CC0905874
:1013A000923048F473DF07C0903829F40FDF03C090
:1013B000911101C09CDF8091E80083FF0AC0E8EE34
:1013C000F0E08081877F8083EBEEF0E080818062B7
:1013D000808308950895CF9380913B01882399F0ED
:1013E000C091E900CF708091EC00982F917080FD42
:1013F00090E8C92B1092E9008091E80083FD9BDF03
:10140000CF70C093E900CF910895E5CF08950F9371
:101410001F93CF93DF93CDB7DEB72A970FB6F8941B
:10142000DEBF0FBECDBF8C011F938F938BE291E087
:101430009F938F93CE0101969F938F93A5D00F908A
:101440000F900F900F900F900F900133110521F422
:1014500085B1806185B906C00233110519F485B1E3
:101460008F7E85B9BE016F5F7F4F80E191E00E9462
:1014700047012A960FB6F894DEBF0FBECDBFDF91AD
:10148000CF911F910F91089584B7877F84BF0FB6C6
:10149000F894A89580916000886180936000109214
:1014A00060000FBE90E080E80FB6F8948093610072
:1014B000909361000FBE84B1806184B9EACC089535
:1014C000E3DF789480E191E00E94B601EC0180E1D5
:1014D00091E00E94E301CD2B09F099DF80E191E0DA
:1014E0000E949E0180E091E0AFD98FDFEBCF08959D
:1014F000089580E091E094D980E191E00E94250177
:10150000E2EEF0E0808184608083089580E191E0E4
:101510000E941B0280E091E030C8089580910E0186
:1015200090910F01009729F0019790930F018093FC
:101530000E0108950F931F9383E090E0F8019183CB
:10154000808381E01F910F91089508950895FB0114
:10155000DC0104C08D910190801921F4415050406C
:10156000C8F7881B990B0895FB01DC0102C00190AC
:101570000D9241505040D8F70895DC0101C06D93A1
:1015800041505040E0F70895AEE0B0E0E9ECFAE0F9
:10159000B6C20D891E8986E08C831A8309838FEF7A
:1015A0009FE79E838D83AE01475E5F4F6F89788D85
:1015B000CE01019608D0EF81F885E00FF11F10826F
:1015C0002E96E4E0B8C2ABE0B0E0E8EEFAE089C203
:1015D0006C017B018A01FC0117821682838181FFE5
:1015E000C0C1CE0101963C01F6019381F70193FD44
:1015F000859193FF81917F01882309F4AEC18532E3
:1016000039F493FD859193FF81917F01853221F417
:10161000B60190E0C1D1E8CF912C212C312CFFE113
:10162000F315E0F08B3279F038F4803279F08332C0
:10163000A9F4232D206110C08D3259F0803371F44C
:10164000232D216009C0832D8260382EE32DE460B4
:1016500022C0F32DF86025C0322E27C037FC2DC0E4
:1016600020ED280F2A3088F436FE06C0892D6AE066
:101670002FD2922E980E19C0822D6AE029D2222EE6
:10168000280E832D8062382E10C08E3231F436FC45
:1016900064C1E32DE0643E2E08C08C3621F4F32DA6
:1016A000F0683F2E02C0883641F4F70193FD859122
:1016B00093FF81917F018111B2CF982F9F7D955427
:1016C000933028F40C5F1F4F2FE329830DC083361E
:1016D00031F0833771F0833509F055C020C0F8012F
:1016E000808189830E5F1F4F88248394912C53013E
:1016F00012C02801F2E04F0E511CF801A080B18009
:1017000036FE03C0692D70E002C06FEF7FEFC501A8
:1017100038D14C018201F32DFF773F2E15C02801EF
:1017200022E0420E511CF801A080B18036FE03C0B9
:10173000692D70E002C06FEF7FEFC50117D14C013A
:10174000F32DF0683F2E820133FC19C0822D90E00A
:1017500088169906A0F4B60180E290E01DD12A9483
:10176000F5CFF50137FC859137FE81915F01B60118
:1017700090E012D121102A9421E0821A910881145C
:10178000910479F7E1C0843611F0893639F5F80112
:1017900037FE07C060817181828193810C5F1F4F8A
:1017A00008C060817181072E000C880B990B0E5FB9
:1017B0001F4FF32DFF763F2E97FF09C09095809520
:1017C000709561957F4F8F4F9F4FF0683F2E2AE0B5
:1017D00030E0A3011DD1882E861844C0853731F42E
:1017E000232D2F7EB22E2AE030E025C0932D997F45
:1017F000B92E8F36C1F018F4883579F0AEC0803735
:1018000019F0883721F0A9C0E92FE061BE2EB4FE9F
:101810000DC0FB2DF460BF2E09C034FE0AC0292F75
:101820002660B22E06C028E030E005C020E130E09E
:1018300002C020E132E0F801B7FE07C0608171818B
:10184000828193810C5F1F4F06C06081718180E0AF
:1018500090E00E5F1F4FA301DBD0882E8618FB2D72
:10186000FF773F2E36FE0DC0232D2E7FA22E89142A
:1018700058F434FE0BC032FC09C0832D8E7EA82E96
:1018800005C0B82CA32C03C0B82C01C0B92CA4FEF1
:101890000FC0FE01E80DF11D8081803321F49A2DE7
:1018A000997EA92E09C0A2FE06C0B394B39404C0C9
:1018B0008A2D867809F0B394A3FC10C0A0FE06C060
:1018C000B21480F4280C922C9B180DC0B21458F45A
:1018D000B60180E290E060D0B394F8CFB21418F46F
:1018E0002B1802C0982C212CA4FE0FC0B60180E357
:1018F00090E052D0A2FE16C0A1FC03C088E790E0A1
:1019000002C088E590E0B6010CC08A2D867851F0BF
:10191000A1FE02C08BE201C080E2A7FC8DE2B6010D
:1019200090E03AD0891430F4B60180E390E034D0EE
:101930009A94F8CF8A94F301E80DF11D8081B601E5
:1019400090E02AD08110F6CF222009F44DCEB601C6
:1019500080E290E021D02A94F7CFF601868197812A
:1019600002C08FEF9FEF2B96E2E1D7C0FC010590FC
:10197000615070400110D8F7809590958E0F9F1F91
:101980000895FC016150704001900110D8F78095D6
:1019900090958E0F9F1F08950F931F93CF93DF9302
:1019A000FB01238121FD03C08FEF9FEF2CC022FF9D
:1019B00016C046815781248135814217530744F46C
:1019C000A081B1819D012F5F3F4F318320838C9394
:1019D000268137812F5F3F4F3783268314C08B01C9
:1019E000EC01FB010084F185E02D0995892BE1F6DE
:1019F000D80116968D919C911797019617969C93F6
:101A00008E931697CE01DF91CF911F910F9108957C
:101A1000FA01AA27283061F1203191F1E8946F93FF
:101A20006E7F6E5F7F4F8F4F9F4FAF4FB1E040D0C3
:101A3000B4E03ED0670F781F891F9A1FA11D680F61
:101A4000791F8A1F911DA11D6A0F711D811D911D96
:101A5000A11D22D009F468943F91062E000C301984
:101A6000000C000C3019305D3193CEF6CF01089593
:101A7000462F4770405D4193B3E00FD0C9F7F6CFD2
:101A8000462F4F70405D4A3318F0495D31FD40529A
:101A9000419302D0A9F7EACFB4E0A6959795879530
:101AA00077956795BA95C9F700976105710508950F
:101AB0009B01AC010A2E06945795479537952795BB
:101AC000BA95C9F7620F731F841F951FA01D089553
:101AD000002480FD060E660F11F08695D1F7802D4B
:101AE00008952F923F924F925F926F927F928F92C2
:101AF0009F92AF92BF92CF92DF92EF92FF920F939D
:101B00001F93CF93DF93CDB7DEB7CA1BDB0B0FB6A6
:101B1000F894DEBF0FBECDBF09942A883988488863
:101B20005F846E847D848C849B84AA84B984C884F9
:101B3000DF80EE80FD800C811B81AA81B981CE0FF0
:101B4000D11D0FB6F894DEBF0FBECDBFED010895D5
:041B5000F894FFCF37
:101B540002810800000134010300000000000000BD
:101B6400008310000001041000000182080000013D
:101B740000000000000000000000006563686F3A88
:041B840025630000D5
:00000001FF
